:100000000C942A000C943F000C943F000C943F0089
:100010000C943F000C943F000C943F000C943F0064
:100020000C943F000C943F000C943F000C943F0054
:100030000C943F000C943F000C943F000C943F0044
:100040000C943F000C943F000C943F000C943F0034
:100050000C943F0011241FBECFE5D8E0DEBFCDBF1A
:1000600010E0A0E6B0E0E4E2F5E002C005900D92F9
:10007000AC3AB107D9F70E9461000C9490020C943D
:10008000000080E487B987E886B9089597B1907E2B
:1000900097B997B18770892B87B9369A349BFECF71
:1000A000349A24B135B1C9010895882349F090E00C
:1000B00020E030E0F9013197F1F79F5F9817D0F316
:1000C0000895CF92DF92EF92FF920F931F93CF93F9
:1000D000DF9380E090E00197F1F780E00E945E01FD
:1000E00081E060E00E94360180E487B987E886B944
:1000F00080E690E00E948F0180E061E00E944A0269
:1001000081E790E00E948F0120E040E050E0CA01CA
:100110000197F1F72F5F2639D1F781E060E00E9467
:10012000360182E890E00E948F0180E061E00E9449
:100130004A0280E990E00E948F0120E040E050E018
:10014000CA010197F1F72F5F2639D1F781E060E00E
:100150000E943601CC24DD2487B1807E87B987B127
:1001600087B9369A349BFECF349A04B115B187B162
:10017000807E87B9389A369A349BFECF349AC4B1C0
:10018000D5B187B1807E87B9399A369A349BFECF34
:10019000349AE4B0F5B080E060E00E944A0281EA5F
:1001A00090E00E948F0102551140B801882777FD29
:1001B0008095982F44E050E00E949F0184EA90E0EF
:1001C0000E948F01C255D140BE01882777FD8095DE
:1001D000982F44E050E00E949F0180E061E00E947F
:1001E0004A0288EA90E00E948F018EEA9EEFE80EB4
:1001F000F91E0027F7FC0095102FC801B70144E055
:1002000050E00E949F0120E0C6010197F1F72F5FA7
:100210002431D1F7A1CF87B3807F87BB969A93987B
:1002200082E08A95F1F722E035E0C49A822F8A9520
:10023000F1F786B38295807F922F9A95F1F7C49853
:10024000932F9A95F1F7C49A922F9A95F1F796B356
:10025000922F9A95F1F7C498932F9A95F1F787FD0D
:10026000E4CF969887B38F6087BB0895282F6623C5
:1002700019F1939A82E08A95F1F7C49A88B3922F84
:1002800092959F70807F982B98BB95E0892F8A95D7
:10029000F1F7C498892F8A95F1F7C49A88B32F7023
:1002A000807F822B88BB892F8A95F1F7C4989A9515
:1002B000F1F70E940B0108959398DCCF1F93182F3C
:1002C0002CE231E040E951E0CA010197F1F72150F9
:1002D0003040D1F787B38F6087BBBC9A8B9A8E9AD8
:1002E00088B3807F88BBC4989698939881E08A955C
:1002F000F1F7C49AC19A85E0982F9A95F1F7C498BE
:100300008A95F1F70E940B0188E260E00E943601B5
:10031000812F8C6060E00E9436011F910895CF9379
:10032000DF93EC018881882339F061E00E94360177
:10033000219688818823C9F7DF91CF9108958F9204
:100340009F92AF92BF92CF92DF92EF92FF920F9364
:100350001F93DF93CF93CDB7DEB727970FB6F894EF
:10036000DEBF0FBECDBF7B018C014A0197FD79C076
:100370008BE261E00E9436015E010894A11CB11C71
:1003800087E0F50111928A95E9F7E114F10401057E
:10039000110519F187E0C82ED12CCC0EDD1EC80145
:1003A000B7012AE030E040E050E00E945302F6013D
:1003B0006083C801B7012AE030E040E050E00E94CD
:1003C0005302C901DA017C018D010894C108D108EA
:1003D000E114F1040105110511F7FFEF8F16FFEF8E
:1003E0009F0689F127E030E02819390927303105C7
:1003F000BCF4F501E20FF31F808189010F5F1F4FED
:100400007501E00EF11E05C0F70181917F010F5FBC
:100410001F4F805D61E00E94360107301105A4F393
:1004200027960FB6F894DEBF0FBECDBFCF91DF91F8
:100430001F910F91FF90EF90DF90CF90BF90AF9002
:100440009F908F9008958981882309F520E030E0FE
:100450002F5F3F4FF501E20FF31F80818823C1F327
:10046000C5CF8DE261E00E94360110950095F094B1
:10047000E094E11CF11C011D111D5E010894A11CFA
:10048000B11C87E0F50111928A95E9F783CF20E04E
:1004900030E0B3CF883230F461118064806860E06E
:1004A0000E943601089597FB092E05260ED057FDB0
:1004B00004D014D00AD0001C38F4509540953095E3
:1004C00021953F4F4F4F5F4F0895F6F790958095D8
:1004D000709561957F4F8F4F9F4F0895A1E21A2E1F
:1004E000AA1BBB1BFD010DC0AA1FBB1FEE1FFF1FD8
:1004F000A217B307E407F50720F0A21BB30BE40B28
:10050000F50B661F771F881F991F1A9469F760956E
:100510007095809590959B01AC01BD01CF01089528
:04052000F894FFCF7D
:100524002020416363656C65726F6D65746572202C
:1005340000202020202020546573742020202020B7
:100544002000202020202065587472656D652000ED
:10055400202020456C656374726F6E69637320207C
:0C05640000583D0020593D005A3D0000A9
:00000001FF
